:020000040000FA
:100000006400F2208613D4200422E8202D307520CD
:10001000FF208620FF203A08B6003B08B70086176D
:100020008620FF203A08B8003B08B90086138620D6
:10003000FF2083164F308600831280200608F300CD
:100040008316403086008312731C3228F31C392833
:10005000731D4328F31D42288613441C5228441064
:100060001422522844140A30F107031C5228F00AC3
:1000700052284414F630F107031C3F28F00AFF30E1
:10008000F00752288617E820FF20E6200B1D4B289A
:10009000003075201928A4013A08A3003B08A200EB
:1000A00017211928E8208620FF203A0803195A282A
:1000B0000B1D5D28003075201928C201DB21D921D4
:1000C000061F6A28C021C208031D7228213075202E
:1000D00020211928C421C208031D72282730752049
:1000E0005521192800307520192883169B001C14EF
:1000F0001A08831203190800922083169B0A772896
:10010000FD30F4006630F5008B28872087207E3094
:10011000F4002030F500F50F8B28F40F8B28003405
:100120000F39303EC003031D9828C100EF2041085D
:100130008616B500350E9D203508F200721C86111A
:1001400072188615F21C0611F2180615721D86101B
:1001500072198614F21D0610F21906140616000014
:1001600006124230F400F40BB32800341830B30008
:10017000BC01BD01BE01BF013C3084000430B400AD
:10018000333080078019F039801B0F398002840AD0
:10019000B40BC028A20DA30DA40DBF0DBE0DBD0D47
:1001A000BC0DB30BBC280800872086120612033052
:1001B0009D20872003309D2003309D2002309D200C
:1001C0000C30F0202830F0200630F0200130EB28F1
:1001D0000930C0000230ED20802886129928C030F6
:1001E000ED20B12806309F00831600309F00373085
:1001F0008100F730850040308600831208000B1123
:100200008101BA01BB018316E73085008720F730F2
:10021000850083120108BA0083160116000001123E
:100220008312BB0301083A0603190C290800B62003
:10023000862188218A218C218E2190219221942946
:10024000430892203C080F3903192C2990208A2159
:100250008C2184218E213F293D0E0F390319362927
:1002600090208C2184218E2190213F293D080F3937
:1002700003194129902084218E219021922111304F
:1002800075283E0E0F39031D4E29203092203E085E
:100290000F39031D4F292030922050298E219021A3
:1002A00092218421942115307528430892203C081E
:1002B0000F390319612990208A2184218C218E21F4
:1002C0006A293D0E0F3903196C29902084218C2155
:1002D0008E219021193075283D080F390319762990
:1002E00090208E2190218421922182293E0E0F3967
:1002F000031D7D29203092207E298E21902184218A
:10030000922194211D3075282E3092283C0E902881
:100310003C0890283D0E90283D0890283E0E9028DD
:100320003E0890283F0E90283F089028AF239B2935
:1003300037239B29E722C2043008A9003108AA000C
:100340003208AB0008002908B0002A08B1002B08C9
:10035000B2002308A9002408AA002508AB00080061
:100360002308A9062906A906A3002408AA062A0626
:10037000AA06A4002508AB062B06AB06A5000800BC
:100380009821F1219A21CF299A21E3219A21F12163
:10039000B0219821F321A3219A21B0219821A41FF3
:1003A000D3292D30D4292030C300A4138B22C204BA
:1003B000B628F721DC29F521F3219821A3219A21E0
:1003C000EB21B0219629A321B830A5006030A4000C
:1003D000FA30A3000800A321A501A401A301013064
:1003E000002A7030F8293630F8293830F8293A30A8
:1003F0008400A321A501A4010008A300840A000829
:10040000A2004A22C204080083163E309B008312D9
:100410000F22F0000D22F100080083169B0A8316BC
:100420001C141A088312080083163E309B007008C3
:100430001E2271081D22831208009B0A9A001C15B7
:1004400055309D00AA309D009C149C18252A8312CB
:100450008C1383160800AF012408031D352A2308D6
:10046000A4000319452AA301AF152F08A502031DF7
:10047000031CA32B0310A41B422AA30DA40DA50B40
:100480003B2AA32BA61FA4130034A401A301A2019D
:10049000A50100349630A500A601A41F582AA20980
:1004A000A309A409A20A0319A30A0319A40AA617F7
:1004B000AF012408031D6D2A2308A4002208A3000D
:1004C000A201AF152408031D6D2A2308A400A3016F
:1004D000AF112F1624080319452A2F08A502031D62
:1004E000031CA32B0310A41B7B2AA20DA30DA40D98
:1004F000A50B732AA32B271B231C422AA21F422AC7
:10050000A30A0319A40A031D422AA40CA30CA50ADA
:1005100003192D2B422AA2012508031900342408AF
:10052000A600A4179630A502A51FDB2AA509A50AD7
:1005300008302502031CB72AA500A20D2308A2003B
:100540002408A300A40108302502031CB72AA50033
:10055000A20D2308A200A30108302502031CB72A1C
:10056000A500A20DA2012508031D0310C02A25081D
:100570000319C02A0310A40CA30CA20CA50BBA2AC1
:10058000271B221CCC2A031CCC2AA20A0319A30A6B
:100590000319A40AA41BDB2AA61F0034A409A3097B
:1005A000A209A20A0319A30A0319A40A0034A40188
:1005B000A301A20100342714A71FFF34A401A61F22
:1005C000FF30A400A300A200A60DA40CFF34250850
:1005D000031D2B080319452A24082A06A6002B0808
:1005E000A5077E30031CF82AA50203182D2BFB2A31
:1005F000A502031CA32B2408A2002308A100A21714
:10060000AA170310A401A3011030AF00211C0E2B68
:100610002908A3072A0803182A0FA407A40CA30C6F
:10062000A20CA10C0310AF0B062BA41B1B2BA20DBD
:10063000A30DA40DA503271B231C2A2BA21F2A2BC5
:10064000A30A0319A40A031D2A2BA40CA30CA50AB0
:1006500003192D2BA61FA4130034A714A71FFF34C2
:10066000FF30A500A400A300A60DA40CFF342B08A6
:100670000319AD2B25080319452A24082A06A600CC
:10068000A417AA17AF012408A2002308A100290873
:10069000A1022A08031C2A0FA202A201A101031C25
:1006A000572B0310A40CA30CA20C0130AF002B0895
:1006B000A502031C612B7E302F07A50703182D2BE5
:1006C000662B7E302F07A507031CA32B1030AE002E
:1006D000A10DA20DA30DA40DAF0D2908A3022A0898
:1006E000031C2A0FA4022A0DAF042F1C792B2114FE
:1006F000802B2908A3072A0803182A0AA407211017
:10070000AE0B682B271B211C9C2B0310A30DA40DE3
:10071000AF0D2908A3022A08031C2A0FA4022A0DE0
:100720002F040139A1070318A20A031D9C2BA20C58
:10073000A10CA50A03192D2BA61FA2132208A400A1
:100740002108A30000342715A71FFF340130A5009E
:10075000A401A301A60DA40CFF34A715FF3480301B
:10076000AA0624082A06AF00A201A80125082B0228
:10077000031CCC2B2B08A0002508AB002008A500EB
:100780002A08A0002408AA002008A4002908A00024
:100790002308A9002008A3002B080319003424080B
:1007A000A600A417AA172B082502AB000319F22BE9
:1007B00008302B02031CE92BAB002908A8002A08EB
:1007C000A900AA0108302B02031CE92B2608A4006B
:1007D00000342B080319F22B0310AA0CA90CA80C47
:1007E000AB0BEC2BAF1FFC2BA809A909AA09A80A7F
:1007F0000319A90A0319AA0A2808A2072908031835
:10080000290FA3072A0803182A0FA407AF1B102CCF
:10081000031C7B2AA40CA30CA20CA50F7B2A2D2B56
:100820000318582AA209A309A409A20A0319A30AB2
:0A0830000319A40A8030A6062B2A43
:02400E00623F0F
:104200002000200020004F00760065007200200092
:10421000520061006E006700650020002000200051
:10422000000020006E0046000000200070004600E4
:10423000000020006D0048000000200075004800CC
:1042400000002000430020003D002000000020006E
:104250004C0020003D002000000020002000200035
:10426000430061006C00690062007200610074002C
:1042700069006E0067002000200000002700100089
:00000001FF
